:100000000C943400189500000C94D9071895000042
:10001000189500001895000018950000189500002C
:10002000189500001895000018950000189500001C
:10003000189500001895000018950000189500000C
:100040000C948E0818950000189500001895000073
:1000500018950000189500001895000018950000EC
:1000600018950000189500008FEF8DBFC8EDE0ECEB
:100070004E2E84E08EBFD4E0F4E05F2EA89584B7C6
:10008000082E877F84BF88E1992780936000909332
:100090006000EEEFF3E0A0E0B1E088278D933197A8
:1000A000E9F70E94FA0D662485E085BD569A80E046
:1000B00084BD7894E99A70916E007E7F70936E0093
:1000C0003B9A3C9A3D9A529A559A569A229825986C
:1000D00053982A9A5B9A2D9A549A5C9A579A209A26
:1000E000219A239824982B9A2C9A3898399A3A98DE
:1000F000409A4198429A80916900837F8093690079
:100100000FEA12E020E030E0A2E4B1E00D931D938D
:100110002D933C93A6E5B1E0EAEEF2E20E94750F62
:100120000CE61DE020E030E0A6E4B1E00D931D9365
:100130002D933C93ABE5B1E0E0EFF2E20E94750F46
:1001400008E316E820E030E0AAE4B1E00D931D9347
:100150002D933C93A0E6B1E0E6EFF2E20E94750F2A
:100160000DE21EE325E030E0AEE4B1E00D931D9317
:100170002D933C93A5E6B1E0ECEFF2E20E94750FFF
:1001800006EC1DE624E330E0A2E5B1E00D931D93FB
:100190002D933C93AAE6B1E0E2E0F3E20E94750FF2
:1001A000A3E9B1E0E8E0F3E20E94750FA7E9B1E04E
:1001B000ECE0F3E20E94750FABE9B1E0E0E1F3E2BD
:1001C0000E94750FAFE9B1E0E4E1F3E20E94750F20
:1001D000A3EAB1E0E8E1F3E20E94750FA7EAB1E01B
:1001E000ECE1F3E20E94750FABEAB1E0E0E2F3E28A
:1001F0000E94750FAFEAB1E0E4E2F3E20E94750FEE
:10020000A3EBB1E0E8E2F3E20E94750FA7EBB1E0E7
:10021000ECE2F3E20E94750F0E94DF0D8CE00E9479
:10022000480E8FE711E00E94EE0DE0E3F3E20E943A
:10023000D80D8FEB11E00E94EE0DE2E4F3E20E9494
:10024000D80DE1E0F0E00E94F10D8FE711E00E948F
:10025000EE0DE4E5F3E20E94D80DE1E0F0E00E944B
:10026000F10D0E94DF0D8FE711E00E94EE0DE6E632
:10027000F3E20E94D80D8FEB11E00E94EE0DE6E74D
:10028000F3E20E94D80DE2E0F0E00E94F10D03B12C
:1002900048E30423A0E8B1E00C9300918001083109
:1002A00011F00C9455010E94F8080E94DF0DE0E067
:1002B000F0E0A4E8B1E00E945511E1E0F0E0AEE02A
:1002C000B1E094E00E945811E5E0F0E0A1ECB1E06B
:1002D0000E945711E7E0F0E0A3ECB1E00E94571153
:1002E000E9E0F0E0A5ECB1E00E94571183E08093D3
:1002F0007F01E2E5F1E00E94CC0F0E94EB0FA3E149
:10030000B1E00E941D10EEEBF2E20E946410E3E106
:10031000F1E00E94CC0F0E942F10EDE0F0E0A3E18D
:10032000B1E00E943811E3E1F1E00E94980FA2E0F1
:10033000B1E0EDE0FF270E943811A2E0B1E00D919D
:100340001D912D913C91A6E0B1E00D931D932D934D
:100350003C93709112017F77709312018FE71CE03C
:100360000E94EE0DECE7F3E20E94D80D81E080934D
:10037000850180918501809386018FEB1DE00E94AD
:10038000EE0DAFE7B1E00D91112745E050E00E947E
:100390006B0FA1E5B1E0A00FB11F0E94D20D00E6E6
:1003A0001BE620E030E0A8E2B1E00D931D932D9311
:1003B0003C93E2E5F1E00E94CC0F0E94EB0FA3E139
:1003C000B1E00E941D1080E08093820180E0809364
:1003D000810100918101093018F011F00C94FA01AB
:1003E0000E94A40CA1E8B1E08C918F5F8C9310F473
:1003F0000C94E90181E0809381010E94A40C70912A
:100400001201777F70931201709112017F7E7093B9
:10041000120181E08093C70181E08093C801A9ECBB
:10042000B1E0E2E8F3E20E94750F0E94DF0D8FE772
:1004300011E00E94EE0DA9ECB1E00E94D20D8FE711
:1004400018E00E94EE0DE8E8F3E20E94D80D5C9AF5
:10045000449845985A9A5D98EF93FF93E0E1F0E055
:100460000E94690EFF91EF915D9A8FEB1DE00E9453
:10047000EE0DAFE7B1E00D91112745E050E00E948D
:100480006B0FA1E5B1E0A00FB11F0E94D20D5D9AE4
:10049000449845985A985C98EF93FF93E0E1F0E018
:1004A0000E94690EFF91EF915C9A82E080930001B7
:1004B0000091850141E0041BA6E3B1E00C9302E04A
:1004C00010E0A6E3B1E04D9155270E94B00DA9E3DD
:1004D000B1E00D931C9330990C949F02449A459A75
:1004E0005A9A5D9A5C98EF93FF93E0E1F0E00E94E6
:1004F000690EFF91EF915C9A419A0091C801013019
:1005000011F00C949D02809184018093830170917D
:100510006E00716070936E00A2E1B1E08C9184FB7B
:1005200016F40C9498027091120178607093120185
:10053000709112017061709312010C94A9020091E4
:10054000C801013018F011F00C94A8020C94A90213
:1005500041980091C801013011F00C94CC03A2E144
:10056000B1E08C9183FB16F00C94CC0300918501D3
:1005700041E0041BA6E3B1E00C9302E010E0A6E327
:10058000B1E04D9155270E94B00DA9E3B1E00D9364
:100590001C93A5ECB1E00D911C91A9E3B1E04D9144
:1005A0005C9104231523ABE3B1E00D931C93009100
:1005B0008501043018F011F00C94E0020C94530300
:1005C000A2E1B1E08C9184FB16F00C941D03ABE327
:1005D000B1E00D911C91003050E0150711F00C9422
:1005E0000703A2E0B1E00D911D912D913C91A8E28D
:1005F000B1E04D915D916D917C910E94C210A2E09D
:10060000B1E00D931D932D933D930C941B03A2E039
:10061000B1E00D911D912D913C91A8E2B1E04D9179
:100620005D916D917C910E94C710A2E0B1E00D93A5
:100630001D932D933D930C945103ABE3B1E00D91C9
:100640001C91003050E0150711F00C943D03A2E01E
:10065000B1E00D911D912D913C91A8E2B1E04D9139
:100660005D916D917C910E94C710A2E0B1E00D9365
:100670001D932D933D930C945103A2E0B1E00D9195
:100680001D912D913C91A8E2B1E04D915D916D914C
:100690007C910E94C210A2E0B1E00D931D932D93B6
:1006A0003D930C94C403A2E1B1E08C9184FB16F459
:1006B0000C949003ABE3B1E00D911C91003050E03D
:1006C000150711F00C947A03A2E0B1E00D911D9191
:1006D0002D913C91A8E2B1E04D915D916D917C919D
:1006E0000E94C210A2E0B1E00D931D932D933D93A3
:1006F0000C948E03A2E0B1E00D911D912D913C91DF
:10070000A8E2B1E04D915D916D917C910E94C7107E
:10071000A2E0B1E00D931D932D933D930C94C4037F
:10072000ABE3B1E00D911C91003050E0150711F0E2
:100730000C94B003A2E0B1E00D911D912D913C917C
:10074000A8E2B1E04D915D916D917C910E94C7103E
:10075000A2E0B1E00D931D932D933D930C94C4033F
:10076000A2E0B1E00D911D912D913C91A8E2B1E084
:100770004D915D916D917C910E94C210A2E0B1E01B
:100780000D931D932D933D9370911201777F70937C
:10079000120182E08093000103B148E30423A0E842
:1007A000B1E00C9300918001003111F00C9407042A
:1007B000A7ECB1E08C918F5F8C930091C701023060
:1007C00018F011F00C94E6030C94E90381E0809397
:1007D000C7018FE711E00E94EE0D0091C7010130C3
:1007E00011F00C94F903A9ECB1E00E94D20D0C9425
:1007F0000104023011F00C940104ECE8F3E20E94D1
:10080000D80D8CE291E00E94750E0C949A06083285
:1008100011F00C945E04A2E1B1E08C9187FB882773
:1008200080F9809580FBA2E1B1E08C9187F98C93EF
:10083000A2E0B1E00D911D912D913C91AAE0B1E0B3
:100840000D931D932D933C93A6E0B1E00D911D9166
:100850002D913C91A2E0B1E00D931D932D933C931B
:10086000AAE0B1E00D911D912D913C91A6E0B1E07F
:100870000D931D932D933C93A2E1B1E08C9187FBE6
:1008800016F00C944D048FE71CE00E94EE0DE4E995
:10089000F3E20E94D80D0C9455048FE71CE00E94EF
:1008A000EE0DECE7F3E20E94D80D82E080930001A8
:1008B0008CE291E00E94750E0C949A06083011F0BB
:1008C0000C9451060091C701013011F00C94C6053B
:1008D000A5E8B1E08C918F5F8C930091850141E098
:1008E000041BA6E3B1E00C9302E010E0A6E3B1E044
:1008F0004D9155270E94B00DA9E3B1E00D931C93D3
:10090000A1ECB1E00D911C91A9E3B1E04D915C9196
:1009100004231523ABE3B1E00D931C93ABE3B1E0EB
:100920000D911C91003050E0150711F00C949A04C1
:100930000C946804009185010A3018F011F00C94B1
:10094000A3040C94A60481E080938501E2E5F1E024
:100950000E94CC0F0E94EB0FA3E1B1E00E941D109A
:1009600000918501013011F00C94C804E2ECF2E230
:100970000E946410E3E1F1E00E94CC0F0E942F106E
:10098000EDE0F0E0A3E1B1E00E9438110C948C0599
:10099000023011F00C94DE04EEEBF2E20E946410DF
:1009A000E3E1F1E00E94CC0F0E942F10EDE0F0E0B7
:1009B000A3E1B1E00E9438110C948C05033011F0D2
:1009C0000C94F404E6ECF2E20E946410E3E1F1E03E
:1009D0000E94CC0F0E942F10EDE0F0E0A3E1B1E007
:1009E0000E9438110C948C05043011F00C940A0507
:1009F000EAECF2E20E946410E3E1F1E00E94CC0F25
:100A00000E942F10EDE0F0E0A3E1B1E00E94381168
:100A10000C948C05053011F00C942005EEECF2E2FC
:100A20000E946410E3E1F1E00E94CC0F0E942F10BD
:100A3000EDE0F0E0A3E1B1E00E9438110C948C05E8
:100A4000063011F00C943605E2EDF2E20E946410DB
:100A5000E3E1F1E00E94CC0F0E942F10EDE0F0E006
:100A6000A3E1B1E00E9438110C948C05073011F01D
:100A70000C944C05E6EDF2E20E946410E3E1F1E033
:100A80000E94CC0F0E942F10EDE0F0E0A3E1B1E056
:100A90000E9438110C948C05083011F00C946205FA
:100AA000EAEDF2E20E946410E3E1F1E00E94CC0F73
:100AB0000E942F10EDE0F0E0A3E1B1E00E943811B8
:100AC0000C948C05093011F00C947805EEEDF2E2EF
:100AD0000E946410E3E1F1E00E94CC0F0E942F100D
:100AE000EDE0F0E0A3E1B1E00E9438110C948C0538
:100AF0000A3011F00C948C05E2EEF2E20E946410D0
:100B0000E3E1F1E00E94CC0F0E942F10EDE0F0E055
:100B1000A3E1B1E00E94381180E0809382010E943D
:100B2000A40C0091850141E0041BA2E8B1E00C9304
:100B30000E94A40C8091850180938601E3E1F1E09D
:100B40000E94980FA2E0B1E0EDE0FF270E9438116B
:100B5000A2E1B1E08C9187FB16F00C94B9058FE708
:100B60001CE00E94EE0DE4E9F3E20E94D80D0C9423
:100B7000C1058FE71CE00E94EE0DECE7F3E20E9456
:100B8000D80D82E0809300010C944B06A8ECB1E0F4
:100B90008C918F5F8C930091C801033018F011F095
:100BA0000C94D4050C94D70581E08093C8015D981E
:100BB000449845985A9A5C98EF93FF93E0E1F0E0EF
:100BC0000E94690EFF91EF915C9A449A45985A9A57
:100BD0005C98EF93FF93E0E1F0E00E94690EFF91D3
:100BE000EF915C9A4498459A5A9A5C98EF93FF93D8
:100BF000E0E1F0E00E94690EFF91EF915C9A8FE7CF
:100C000018E00E94EE0D0091C801013011F00C9423
:100C10001D06E8E8F3E20E94D80D5D9A44984598D5
:100C20005A9A5C98EF93FF93E0E1F0E00E94690E1E
:100C3000FF91EF915C9A0C944B06023011F00C94EA
:100C40003506EAE9F3E20E94D80D5D9A449A459888
:100C50005A9A5C98EF93FF93E0E1F0E00E94690EEE
:100C6000FF91EF915C9A0C944B06033011F00C94B9
:100C70004B06EEE9F3E20E94D80D5D9A4498459A3E
:100C80005A9A5C98EF93FF93E0E1F0E00E94690EBE
:100C9000FF91EF915C9A8CE291E00E94750E0C94AA
:100CA0009A06003311F00C946F068FE71CE00E9447
:100CB000EE0DE2EAF3E20E94D80DA2E0B1E00D9160
:100CC0001D912D913C91A6E0B1E00D931D932D93C4
:100CD0003C938CE291E00E94750E0C949A060032CF
:100CE00011F00C949A06AFE7B1E08C918F5F8C9372
:100CF00000917F01083018F011F00C9481060C94DB
:100D0000840681E080937F018FEB1DE00E94EE0D51
:100D1000AFE7B1E00D91112745E050E00E946B0F65
:100D2000A1E5B1E0A00FB11F0E94D20D8CE291E0CD
:100D30000E94750E00910001003018F011F00C9423
:100D4000A3060C94D50700910001023011F00C9419
:100D5000BF07A2E0B1E00D911D912D913C91AAE059
:100D6000B1E00D931D932D933C93A3ECB1E00D9155
:100D70001C91A9E3B1E04D915C9104231523ABE3F1
:100D8000B1E00D931C93ABE3B1E00D911C910030E9
:100D900050E0150718F011F00C94D0060C943E07A3
:100DA000A5ECB1E00D911C91A9E3B1E04D915C91EE
:100DB00004231523ADE3B1E00D931C93ADE3B1E043
:100DC0000D911C91003050E0150718F011F00C94B3
:100DD000EB060C940107A2E0B1E00D911D912D915D
:100DE0003C91AEE0B1E04D915D916D917C910E949E
:100DF000C210A2E0B1E00D931D932D933D930C948E
:100E00003E07AEE0B1E04D915D916D917C91A2E025
:100E1000B1E00D911D912D913C9104171507260706
:100E2000370710F40C942A07A2E0B1E00D911D9150
:100E30002D913C91AEE0B1E04D915D916D917C9131
:100E40000E94C710A2E0B1E00D931D932D933D9336
:100E50000C943E07AEE0B1E00D911D912D913C91B7
:100E6000A2E0B1E04D915D916D917C910E94C7101F
:100E7000A2E0B1E00D931D932D933D935A924A92B7
:100E8000A2E0B1E00D911D912D913C91D2010D9305
:100E90001D932D933C9384E00E94670F0E94210DC7
:100EA000229684E00E948A0DAAE0B1E00D911D9186
:100EB0002D913C91A2E0B1E00D931D932D933C93B5
:100EC000E2E0F1E00E94CC0F0E94EB0FA3E1B1E061
:100ED0000E941D10E6EEF2E20E946410E3E1F1E0F0
:100EE0000E94CC0F0E942F10EDE0F0E0A3E1B1E0F2
:100EF0000E943811A8EAB4E0AF93BF93E3E1F1E0B8
:100F00000E94CC0F0E94840E11E005E0BF91AF91CA
:100F10000E947A10E8EAF4E0A7E1B1E00E94331100
:100F20008FEB11E00E94EE0DE8EAF3E20E94D80D8B
:100F30008FEB11E00E94EE0DA7E1B1E00E94D20D0F
:100F4000E6EBF3E20E94D80DA2E1B1E08C9187FBC1
:100F500016F00C94B5078FE71CE00E94EE0DE4E953
:100F6000F3E20E94D80D0C94BD078FE71CE00E94AD
:100F7000EE0DECE7F3E20E94D80D0C94D1078FEB55
:100F80001DE00E94EE0DAFE7B1E00D91112745E0A5
:100F900050E00E946B0FA1E5B1E0A00FB11F0E94CD
:100FA000D20D80E080930001E99A0C946B02F894D2
:100FB000FFCF0F921F922F923F924F925F927F929C
:100FC000AF92BF920F931F932F933F934F935F93D3
:100FD0006F937F938F939F93AF93BF93CF93DF9341
:100FE000EF93FF938FB78F93E99882E090E00E9490
:100FF000750E03B148E30423A0E8B1E00C9300911F
:101000008001083111F00C942E081A9B0C941B08D7
:10101000AFE7B1E08C918F5F8C9300917F01053039
:1010200018F011F00C9416080C94190881E08093C4
:101030007F010C94290880917F01815080937F016A
:1010400000917F01003011F00C94290885E0809315
:101050007F0181E0809300010C9472081A9B0C942C
:101060005108A2E0B1E00D911D912D913C91AFE7A7
:10107000B1E0AD90BB24AEE3B1E0AA0CBB1CAA0C5E
:10108000BB1CAA0DBB1D4D915D916D917C910E9481
:10109000C210A2E0B1E00D931D932D933D930C94EB
:1010A0006F08A2E0B1E00D911D912D913C91AFE749
:1010B000B1E0AD90BB24AEE3B1E0AA0CBB1CAA0C1E
:1010C000BB1CAA0DBB1D4D915D916D917C910E9441
:1010D000C710A2E0B1E00D931D932D933D9382E0E4
:1010E000809300018F918FBFFF91EF91DF91CF919E
:1010F000BF91AF919F918F917F916F915F914F9130
:101100003F912F911F910F91BF90AF907F905F9073
:101110004F903F902F901F900F9018950F921F9215
:101120002F923F924F925F927F92AF92BF920F9316
:101130001F932F933F934F935F936F937F938F935F
:101140009F93AF93BF93CF93DF93EF93FF938FB7AB
:101150008F93A3E8B1E08C9181508C93009183012F
:10116000003011F00C94DC08419880918401809348
:10117000830180E08093820187E0809381017091F8
:101180006E007E7F70936E00709112017F7E70936F
:10119000120170911201786070931201449A459A7D
:1011A0005A9A5D985C98EF93FF93E0E1F0E00E941B
:1011B000690EFF91EF915C9A8F918FBFFF91EF9134
:1011C000DF91CF91BF91AF919F918F917F916F915F
:1011D0005F914F913F912F911F910F91BF90AF90D1
:1011E0007F905F904F903F902F901F900F90189599
:1011F000E0E0F0E0A4E8B1E00E945511E1E0F0E0A9
:10120000AEE0B1E094E00E945811E5E0F0E0A1EC1E
:10121000B1E00E945711E7E0F0E0A3ECB1E00E94DA
:101220005711E9E0F0E0A5ECB1E00E94571181E030
:101230008093360100913601033018F011F00C94C0
:1012400023090C94260981E08093360184EF91E014
:101250000E94750E00913601013011F00C94A20924
:101260000E94DF0D8FE711E00E94EE0DECEBF3E240
:101270000E94D80D8FEB11E00E94EE0DE4ECF3E23A
:101280000E94D80D8FEB16E00E94EE0DA8EAB4E0A4
:10129000E4E8F1E00E94E9100E94D00D03B148E3B8
:1012A0000423A0E8B1E00C9300918001083011F014
:1012B0000C945E090E94DF0D0C949B090091800143
:1012C000003311F00C946D0980918401815080935A
:1012D00084018AEF90E00E94750E00918001003237
:1012E00011F00C947C09A4E8B1E08C918F5F8C9391
:1012F0008AEF90E00E94750E009184010C3318F083
:1013000011F00C9485090C9488098CE38093840176
:1013100000918401013010F00C94910981E08093D8
:10132000840100918001083211F00C9499090C9409
:10133000490C0C943209A6E3B1E08C918F5F8C9339
:101340000C94470C023011F00C945A0A0E94DF0DE5
:101350008FE711E00E94EE0DE4EDF3E20E94D80D5C
:101360008FEB1DE00E94EE0DAFE7B1E00D9111276C
:1013700045E050E00E946B0FA1E5B1E0A00FB11F66
:101380000E94D20DAEE0B1E00D911D912D913C91E6
:10139000A2E0B1E00D931D932D933C9382E08093E6
:1013A000000103B148E30423A0E8B1E00C930091ED
:1013B0008001083011F00C94E1090E94DF0D0C94BB
:1013C000530A00918001083211F00C94E9090C9441
:1013D000490C00910001003018F011F00C94F20952
:1013E0000C94510A00910001023011F00C943E0A55
:1013F000E2E0F1E00E94CC0F0E94EB0FA3E1B1E02C
:101400000E941D10E6EEF2E20E946410E3E1F1E0BA
:101410000E94CC0F0E942F10EDE0F0E0A3E1B1E0BC
:101420000E943811A8EAB4E0AF93BF93E3E1F1E082
:101430000E94CC0F0E94840E11E005E0BF91AF9195
:101440000E947A10E8EAF4E0A7E1B1E00E943311CB
:101450008FEB11E00E94EE0DE8EAF3E20E94D80D56
:101460008FEB11E00E94EE0DA7E1B1E00E94D20DDA
:10147000E6EBF3E20E94D80D0C94500A8FEB1DE0CE
:101480000E94EE0DAFE7B1E00D91112745E050E06D
:101490000E946B0FA1E5B1E0A00FB11F0E94D20D19
:1014A000E99A0C94D109A6E3B1E08C918F5F8C93FB
:1014B0000C94470C033011F00C94470C81E080939E
:1014C000370181E0809338010E94DF0D8FE711E042
:1014D0000E94EE0DE0EEF3E20E94D80DA7E3B1E02A
:1014E0000D91112744E050E00E946B0FAFE8B1E08E
:1014F000A00FB11F0E94D20DECEEF3E20E94D80DB6
:10150000A7E3B1E00D91112741E050E0041B150B5A
:10151000A9E3B1E00D931C9302E010E0A9E3B1E070
:101520004D915C910E94B00DA9E3B1E00D931C9325
:10153000A1ECB1E00D911C91A9E3B1E04D915C915A
:1015400004231523ABE3B1E00D931C930FEF13E0DD
:10155000ABE3B1E04D915C91041B150BADE3B1E041
:101560000D931C93ABE3B1E00D911C91003050E062
:10157000150718F011F00C94BF0A0C94C70AABEBD6
:10158000B1E0E0EFF3E20E94750F0C94D20AABEBEE
:10159000B1E0E4EFF3E20E94750F81E0809338013F
:1015A0000C94370BA3ECB1E00D911C91A9E3B1E0D1
:1015B0004D915C9104231523ABE3B1E00D931C9393
:1015C000ABE3B1E00D911C91003050E0150718F02D
:1015D00011F00C94ED0A0C94F70AABEBB1E00E9409
:1015E000C90DEAEFF3E20E94750F0C94040BABEB0C
:1015F000B1E00E94C90DEEEFF3E20E94750F82E0A8
:10160000809338010C94370BA5ECB1E00D911C913F
:10161000A9E3B1E04D915C9104231523ABE3B1E064
:101620000D931C93ABE3B1E00D911C91003050E0A1
:10163000150718F011F00C941F0B0C942C0BABEB4E
:10164000B1E00E94C90DE2E0F4E20E94750F83E070
:10165000809338010C94370BABEBB1E00E94C90DBD
:10166000E4E0F4E20E94750F84E0809338018FEB90
:1016700011E00E94EE0DE6E0F4E20E94D80DABEB23
:10168000B1E00E94D20D03B148E30423A0E8B1E029
:101690000C9300918001083011F00C94530B0E94C0
:1016A000DF0D0C94420C00918001083111F00C9474
:1016B0006E0BA7E3B1E08C918F5F8C9300913701A3
:1016C0000A3018F011F00C94670B0C946A0B81E04F
:1016D000809337018AEF90E00E94750E009180019F
:1016E000003311F00C94860B809138018150809367
:1016F000380100913801013010F00C94820B84E025
:10170000809338018AEF90E00E94750E009180016D
:10171000003211F00C94A10BA8E3B1E08C918F5F23
:101720008C9300913801043018F011F00C949A0B4E
:101730000C949D0B81E0809338018AEF90E00E9429
:10174000750EA1ECB1E00D911C91ADE3B1E04D91AE
:101750005C9104231523A1ECB1E00D931C93A3EC41
:10176000B1E00D911C91ADE3B1E04D915C9104238A
:101770001523A3ECB1E00D931C93A5ECB1E00D9102
:101780001C91ADE3B1E04D915C9104231523A5ECD0
:10179000B1E00D931C9300913801013011F00C94CD
:1017A000D40B00000C94380C023011F00C94E80BB0
:1017B000A1ECB1E00D911C91A9E3B1E04D915C91D8
:1017C000040F151FA1ECB1E00D931C930C94380C81
:1017D000033011F00C94180CA1ECB1E00D911C91A8
:1017E000A9E3B1E04D915C91040F151FA1ECB1E0AC
:1017F0000D931C93A3ECB1E00D911C91A9E3B1E012
:101800004D915C91040F151FA3ECB1E00D931C9357
:10181000A5ECB1E00D911C91A9E3B1E04D915C9173
:10182000040F151FA5ECB1E00D931C930C94380C1C
:10183000043011F00C94380CA1ECB1E00D911C9126
:10184000A9E3B1E04D915C91040F151FA1ECB1E04B
:101850000D931C93A3ECB1E00D911C91A9E3B1E0B1
:101860004D915C91040F151FA3ECB1E00D931C93F7
:1018700000918001083211F00C94400C0C94490C3A
:101880000C94660AA6E3B1E08C918F5F8C930C9464
:101890001A090E94DF0DE2E1F4E20E94D80DE0E0B7
:1018A000F0E0A4E8B1E07BE70E944411E1E0F0E061
:1018B000A2E0B1E094E07BE70E944711E5E0F0E0B0
:1018C000A1ECB1E07BE70E944611E7E0F0E0A3EC79
:1018D000B1E07BE70E944611E9E0F0E0A5ECB1E061
:1018E0007BE70E944611E1E0F0E00E94F10D0895CF
:1018F0000895289A81E08093D0010091D0010830AA
:1019000018F011F00C948E0C5F9A5F98A0EDB1E086
:101910008C918F5F8C9310F40C947D0C289881E04F
:101920008093D0010091D001083018F011F00C9490
:10193000A30C5F9A5F98A0EDB1E08C918F5F8C93C0
:1019400010F40C94920C08958FE715E00E94EE0DB0
:10195000449845985A980091820141E00423A1EDF2
:10196000B1E00C930091D101013011F00C94BB0C4B
:101970005D9A0C94BC0C5D985C98EF93FF93E0E14A
:10198000F0E00E94690EFF91EF915C9A449A4598AD
:101990005A980091820142E00423A1EDB1E00C933A
:1019A0000091D101023011F00C94D90C5D9A0C9485
:1019B000DA0C5D985C98EF93FF93E0E1F0E00E9411
:1019C000690EFF91EF915C9A4498459A5A9800915C
:1019D000820144E00423A1EDB1E00C930091D10118
:1019E000043011F00C94F70C5D9A0C94F80C5D988F
:1019F0005C98EF93FF93E0E1F0E00E94690EFF91A5
:101A0000EF915C9A449A459A5A980091820148E075
:101A10000423A1EDB1E00C930091D101083011F045
:101A20000C94150D5D9A0C94160D5D985C98EF93CF
:101A3000FF93E0E1F0E00E94690EFF91EF915C9A64
:101A40000895289881E08093D2010091D20100325C
:101A500018F011F00C94530D00274427A881B98188
:101A60008C9180FB00F94160042300FBA2E1B1E00E
:101A70008C9182F98C93A2E1B1E08C9182FBA5E27A
:101A8000B0E08C9181F98C935F9A5F9891E0A88186
:101A9000B9810E94850FA2EDB1E08C918F5F8C938C
:101AA00010F40C94250D81E08093D2010091D201B5
:101AB000083018F011F00C94840D00274427A1E0A1
:101AC000B1E08C9180FB00F94160042300FBA2E1AE
:101AD000B1E08C9182F98C93A2E1B1E08C9182FB10
:101AE000A5E2B0E08C9181F98C935F9A5F9891E0C8
:101AF000A1E0B1E00E947B0FA2EDB1E08C918F5F7D
:101B00008C9310F40C94560D289A28980895481A2E
:101B1000590A0895481A8827580A089505D00E943E
:101B20006B0F00FC0CD008950024E89457FF02C00E
:101B300009D0689400F80BD010F80124089502D061
:101B400009D00895509540954F5F5F4F0895E894F0
:101B500017FF0895009510950F5F1F4F6894089523
:101B600014D081F0002E112E415050400ED009F4B7
:101B700008954F935F93402D512D0E946B0F5F91FD
:101B80004F91F2CF01E0112708958827842B852BF0
:101B900008958F938D918823E9F711978F91089578
:101BA000A8EAB4E08D91882311F06CD0FBCF0895A2
:101BB0000E946010802D11F065D0FACF089581E069
:101BC00067D015D080E864C08FE7213039F08FEB03
:101BD000223021F08FE8233009F08FEC810F0C9434
:101BE000480E88EE93E081D03197D9F7089583E0CD
:101BF00099277BC08AEF90E00E94750E559A529A01
:101C00003D9A3C9A3B9A569A5E9885E090E00E94F5
:101C1000750E43985D985A98459A449A439AEF9363
:101C2000FF93E4ECF0E00E94690EFF91EF9143987E
:101C300059D0439AEF93FF93E4ECF0E00E94690ED1
:101C4000FF91EF9143984ED0439AEF93FF93E4ECCA
:101C5000F0E00E94690EFF91EF91439843D04498C1
:101C6000439AEF93FF93E4ECF0E00E94690EFF913A
:101C7000EF91439837D088E20BD08EE009D086E010
:101C800007D008955E9A829505D004D02BD0089590
:101C90005E98F9CF859510F4449A01C044988595D3
:101CA00010F4459A01C04598859510F45A9A01C0E0
:101CB0005A98859510F45D9A01C05D98439AEF9308
:101CC000FF93E4ECF0E00E94690EFF91EF914398DE
:101CD00008953197F1F70895689462F80895E894AB
:101CE00062F8089581E090E000C0EF93FF93EE2743
:101CF000E82BE92B31F0E0EDF7E03197F1F70197B0
:101D0000D1F7FF91EF9108958DE207FD8D938F2D0F
:101D1000881F802F881F8F57082F6894F7F8802F0F
:101D200087FF15C080958395082F80E38D938EE201
:101D30008D93802F815228F080E38D9399279C9377
:101D4000089544270A95802F09F196D01FC080522C
:101D500030F09EE49D9381E48D939D93EFCF4427D3
:101D6000DF92EF92FF920F938FE1801B11F0082F0B
:101D700083D089D09EE29D930F91FF90EF90DF90EA
:101D800044270395003209F4D7CF2BD03F93E8E1E5
:101D9000FEE138E12F2D1E2D0D2DFF24EE24DD2434
:101DA0004427000F111F221FA8F42F923F920E9478
:101DB0006010102C0E946010202C0E946010302CAB
:101DC0000E9460103197410DD21CE31CF01C3F9023
:101DD0002F9001C0339631963A9519F73F9107D06D
:101DE000AFCFDD0CEE1CFF1C0A95D9F70895002734
:101DF00019E058D08F93802B11F0039501C08F917B
:101E00001A95B9F7802F882309F496CF8F91805DBA
:101E10008D930A95D9F792CF0065CD1D80B2E60E5D
:101E200040597307A0ACB90350D6DC01286BEE0013
:101E300094357700CA9A3B0065CD1D00B2E60E00CE
:101E400059730700ACB90300D6DC01006BEE00004B
:101E5000357700009A3B0000CD1D0000E60E000023
:101E600073070000B9030000DC010000EE00000071
:101E7000770000003B000000F694E794D794479564
:101E80000A95D1F7089500270DD08F9303958F2DD4
:101E90008E298D29842BC1F78F91805D8D930A95B2
:101EA000D9F74CCF1F930F93002710E2440FDD1C8E
:101EB000EE1CFF1C001F802F9AE0890B10F0082FEA
:101EC00043951A9599F7802F0F911F910895480E09
:101ED0008827581E08950F92B801469F8001479F9A
:101EE000100D569F100D0F9008950E9460100D92D6
:101EF0000020D9F70895903039F08C91869508F438
:101F000080689A95D9F78C930895903081F00D915F
:101F10001D912D913C91369527951795079508F4BD
:101F200030689A95C1F73C932E931E930E930895B3
:101F300033D0992711278F2D880F80E8F82A802F1A
:101F4000881F08F41FEF41F08F57082F07FD04C0CA
:101F5000003240F08FEF01C08827982FD82EE82E4E
:101F6000F82E09C08FE1801B082FF694E794D794D0
:101F700097950A95D1F7112351F09095D094E0945C
:101F8000F09481E0980F8827D81EE81EF81E0F2DC8
:101F9000FE2CED2CD92E0895D190E190F190019175
:101FA0000895102F90E8FF0C001F0927990FF79450
:101FB0001078652F90E8440F551F5927990F4795C2
:101FC000607800380895FF0C90E89027110F9795DE
:101FD000F794092F0895102FBD2CDE2CEF2CF02E36
:101FE00011234AF4B094D094E094F0949FEFB91A7E
:101FF000D90AE90AF90A0EE1FF2039F4FE2CED2C8A
:10200000DB2CBB240850C2F724C032F00A95BB0C6D
:10201000DD1CEE1CFF1CF9CF0E940F10D4CFB7FEC1
:10202000089590E8B91611F4D0FE08959FEFD91ADB
:10203000E90AF90A09F403950895DD92ED92FD92FB
:102040000C9308959FE7092FF92A9FEFD92EE92EC7
:102050000895DD24EE24FF24002711270895A1DF31
:10206000C1F35038B1F31627005850580894051F93
:1020700012F418F4E7CF08F0ECCF0BD0FF202AF0D1
:10208000BB0CDD1CEE1CFF1C9ECF0F5F0BF4DACFE8
:102090009ACF9F929924AA24BB24992788E1990C6E
:1020A000AA1CBB1CDD1CEE1CFF1C30F4920EA31EF0
:1020B000B41ED91EE91EF91E8A9589F79F900895CE
:1020C000C895319600200895FBDF202DF9DF302DD3
:1020D000F7DF402DF5DF502D089599278D919395C9
:1020E0008823E1F7939511968C9311978E919A9589
:1020F000D1F70895EA2FFB2F00244C918D91039482
:102100008E32E1F711248D9113948823E1F71A940C
:10211000101640F41197202F2119239580E38D93F9
:102120002A95E9F7113039F59927AE2FBF2FA00D69
:10213000B91FA00FB91F8C919C93853308F421C05F
:1021400031E08E918E32E9F38D3241F0830F8A3384
:1021500019F480E331E001C033278C93AE1789F77F
:10216000332341F0AE2FBF2FB8DF81E34D3209F4A6
:102170003196808308958827E00DF81FE00FF81F3F
:1021800080830895040F151F261F371F0895041B11
:10219000150B260B370B0895000F111F221F331F3D
:1021A000089500951095209530950F5F1F4F2F4F84
:1021B0003F4F0895019110810EC00191119121911D
:1021C00030810BC00191108117FF05C03FEF2FEF49
:1021D00004C0008111272227332737FF03C0E1DF26
:1021E0008DE28D93CF93DF93CF92DF92EF92AA246B
:1021F000BB24CC24DD24EE2440E2CAE0DD2755E0F8
:1022000093E38881890F87FD9F7083FD907F891BF1
:1022100089935A95A9F7C0DFAA1CBB1CCC1CDD1CF6
:10222000EE1C4A9551F7E894EFE0FF2782910ED01B
:10223000EB30E0F71EF068948A2D0CD088278D9340
:10224000EF90DF90CF90DF91CF910895982F8295F6
:1022500001D0892F8F70805D26F0803309F40895B6
:1022600068948D93089581918D938823E1F7089563
:1022700094E081918D939A95E1F70895F999FECFB5
:10228000E1BDF2BD3196089591E001C092E07B3747
:1022900051F47FB7F894F2DF8D9180BDFA9AF99AE4
:1022A0009A95C9F77FBF7727089591E001C092E022
:1022B000E5DFF89A80B58D939A95D1F708950000DF
:1022C0000C420000904100008C420000CA42000015
:1022D0000C43299C34430000524366E678430000D7
:1022E0008C430000FA430000FA323230487A000092
:1022F000313030480000316B487A00002031306BBB
:1023000000003130306B0000312E3800332E3500A4
:10231000372E300020313000203134002031380099
:102320002032310020323400203238002035300095
:1023300020535036465245204444532D6269732041
:102340000000687474703A2F2F6C782D6E65742EAF
:10235000706C0000202020207665722E20312E31F6
:1023600061202020000050726573732062757474C0
:102370006F6E20746F005345545550004631202035
:1023800020002A5452582A00435720004D6F64659C
:10239000202000004632202020004C53420055539C
:1023A000420046313D4632002020202020202020BF
:1023B0002020202000004D487A2000004357206450
:1023C000656C000044656C3D202020202A203330BD
:1023D0006D73000055737461772E20466D6964003B
:1023E0005061736D6F202020202000004D487A003E
:1023F000412000004E20582058004D200000302081
:1024000058002B002D005374616E202020202020C6
:0824100020005A61706973009D
:00000001FF
